:060000000A128A11122809
:10000800FE00030EF3000408F4000A08F50083124A
:1000180003137F08F6000A128A111F2B0A128A118D
:100028001528F001F101F801F901FA01FB01831328
:10003800203084003D300A128A11322483010A12CA
:100048008A1126288B01831203139F010630831619
:1000580003139F008501831203138501C0308316A3
:1000680003138600C030831203138600BF30831643
:10007800031387003F30831203138700043083166D
:100088000313810083120313A8017D30C4004408C0
:10009800C800A701A001F901F801A201A101A60168
:1000A800A501F111F0127013F0137110F110711114
:1000B800FB01A401F0117011FA010030BD000030FD
:1000C800BE001430BF000030C00029300A128A1167
:1000D800CE230A128A11F010701283120313A3019F
:1000E8007010051070150A128A11EF230A128A116E
:1000F80006308312031381008B160B178316031324
:100108008C168B17FB080319FA0114307A02031CAA
:10011800BF287011F011FA018312C701C60113300C
:1001280046020318B4284608293E840083130008B1
:10013800C4004408BD004608013E0A128A1103247F
:100148000A128A11831203134707C5004508C7001E
:100158000130C4004408C60713304602031C972820
:100168003C084706031DBE282908493A031DBE2836
:10017800F014BF287015F01C922AF01083122B0877
:10018800C13A031DCC28C230C4004408AB00152A6C
:100198002B08013A031DD228280809292B08023AFE
:1001A800031D0D29C701F01EDE2847080138C400C9
:1001B8004408C700701FE52847080238C4004408EF
:1001C800C700F01FEC2847080438C4004408C700DB
:1001D800711CF32847080838C4004408C700F11CFC
:1001E800FA2847081038C4004408C700711D0129BF
:1001F80047082038C4004408C700F11D08294708EB
:100208008038C4004408C7004708C4004408AC004C
:10021800152A2B08413A031D1B29C230C400440883
:10022800AB000A128A1116240A128A11152A83129F
:1002380003132B08423A031D2B29C230C40044087B
:10024800AB000A128A1124240A128A11152A831271
:1002580003132B08493A031D3729C230C400440848
:10026800AB00F016152A2B084A3A031D4129C23063
:10027800C4004408AB007017152A2B084B3A031D1D
:100288004B29C230C4004408AB00F017152A2B08CC
:100298004C3A031D5529C230C4004408AB00711400
:1002A800152A2B084D3A031D5F29C230C4004408A3
:1002B800AB00F114152A2B084E3A031D6829C230E9
:1002C800C4004408AB0075292B084F3A031D772951
:1002D800C230C4004408AB00F0167017F017711450
:1002E800F1147115152A2B08513A031D8129C230C2
:1002F800C4004408AB00F012152A2B08523A031D1B
:100308008B29C230C4004408AB007013152A2B088F
:10031800533A031D9529C230C4004408AB00F013BA
:10032800152A2B08543A031D9F29C230C4004408DB
:10033800AB007110152A2B08553A031DA929C230A4
:10034800C4004408AB00F110152A2B08563A031DC7
:10035800B229C230C4004408AB00BF292B08573A61
:10036800031DC129C230C4004408AB00F012701349
:10037800F0137110F1107111152A2B08593A031D49
:10038800CC29C230C4004408AB002030F006152A3E
:100398002B085A3A031DD729C230C4004408AB00C1
:1003A8004030F006152A2B085B3A031DE229C230BB
:1003B800C4004408AB008030F006152A2B085C3ACC
:1003C800031DED29C230C4004408AB000130F1061A
:1003D800152A2B085D3A031DF829C230C4004408C9
:1003E800AB000230F106152A2B085E3A031D012ADC
:1003F800C230C4004408AB00132A2B085F3A031D1F
:10040800162AC230C4004408AB002030F006403041
:10041800F0068030F0060130F1060230F1060430B3
:10042800F1067016701E902A7012831203132A08A0
:10043800C4004408A9004930C4004408AA00C70100
:10044800C601133046020318462A4608293E84008E
:1004580083130008C4004408BD004608013E0A1280
:100468008A1103240A128A11831203134707C5004D
:100478004508C7000130C4004408C60713304602C7
:10048800031C292A4708C4004408BC000A30C400D9
:100498004408C700602AC7080319632AF0110D3001
:1004A800C500FB30C400C40B572AC50B572A5C2A69
:1004B800013083120313C702F0194F2A7014701CFD
:1004C800902A70100430C4004408A4000514C60122
:1004D8001430460203188E2A4608293E84008313E6
:1004E800000899000230C4004408FB008316031377
:1004F8009818812AFB08031D7A2AFB0803198E2AFB
:10050800013083120313C4004408C607143046029E
:10051800031C702A83120510FA01701578088312DB
:10052800031322060319D42A78081F3A031DA12AA7
:100538000A128A1116240A128A117808203A031D11
:10054800AA2A0A128A1124240A128A117808293A36
:10055800031DB02A2030F00678082A3A031DB62A6F
:100568004030F00678082B3A031DBC2A8030F0068C
:1005780078082C3A031DC22A0130F10678082D3A72
:10058800031DC82A0230F10678082E3A031DCE2A28
:100598000430F106780883120313C4004408A2004B
:1005A800A6080319DB2A831203138514DE2A831293
:1005B80003138510A5080319E52A831203130515EB
:1005C800E82A831203130511F01EEE2A831203137F
:1005D8000614F12A831203130610701FF72A8312D8
:1005E80003138614FA2A831203138610F01F002BB4
:1005F800831203130615032B831203130611711CB0
:10060800092B8312031386150C2B831203138611EF
:10061800F11C122B831203130616152B83120313D6
:100628000612711D1B2B831203138616862883124C
:100638000313861286280B1D962B0B11063081009A
:100648000130C802C808031D3B2B7D30F200720838
:10065800C8000430F2007208A70026080319362BD8
:100668000130A602250803193B2B0130A5022708F3
:100678000319422B0130A7028516432B85127B08EC
:100688000319482B0130FB02200803194D2B0130B8
:10069800A002A008031D962BF901061B572B1F303B
:1006A800F2007208F900861B5D2B2030F2007208F8
:1006B800F9000718632B2930F2007208F90087182F
:1006C800692B2A30F2007208F90007196F2B2B30BA
:1006D800F2007208F9008719752B2C30F2007208A5
:1006E800F900071A7B2B2D30F2007208F900871ADF
:1006F800812B2E30F2007208F90079082106031DBB
:100708008A2B7908F2007208F800962B7908F20013
:100718007208A100F80178080319962B0630F20038
:100728007208A0008C1EC32B0230F2007208FB0076
:100738008C129818A12B181DAC2B981CA52B1812DD
:100748001816181DC32B1A08F2007208F700C32BDD
:10075800F0151A08F2007208F700701DC32B143048
:100768007A020318C32B7708F2007A08293E84001E
:100778007208831380000130F2007208FA077608C5
:10078800FF0075088A0074088400730E8300FE0E4B
:100798007E0E090083120313C2004208C1004108FB
:1007A800C3000130BF020030031CC003C002FF3089
:1007B8004006031DE12BFF303F06031908003D08E2
:1007C800C100430884004108831380000130C10040
:1007D8004108C307D52B8316031318150C3099004D
:1007E8001812831203139817181383160313181378
:1007F800831203131816831603139816080083121E
:100808000313C000BF01401C0D2C3D08BE003E086C
:10081800BF070310BD0D0310C00CC008031D072C33
:100828003F080800F115F0127013F0137110F11061
:100838007111023083120313BD003D08A6000800A1
:10084800F111F0127013F0137110F11071110230E0
:1008580083120313BD003D08A50008006400800151
:0C086800840A0406031900340406332C33
:02400E0071FF40
:00000001FF
